:100000000C9437000C945F000C945F000C945F001C
:100010000C945F000C945F000C945F000C947003D0
:100020000C945F000C945F000C945F000C945F00D4
:100030000C945F000C945F000C945F000C945F00C4
:100040000C945F000C945F000C945F000C945F00B4
:100050000C945F000C945F000C945F000C945F00A4
:100060000C945F000C945F00C8006903E404112441
:100070001FBECFEFD4E0DEBFCDBF11E0A0E0B1E006
:10008000E6ECF2E102C005900D92AA33B107D9F770
:1000900012E0AAE3B1E001C01D92AA31B107E1F775
:1000A00010E0CEE6D0E004C02297FE010E945E0977
:1000B000C836D107C9F70E94C4010C9462090C9498
:1000C0000000E1EBF1E0A8EBB1E08C912081820F20
:1000D000912D911D9695879580833197119781E099
:1000E000EA3AF80791F708950F931F93019709F0E3
:1000F0004CC06F5F7F4F09F048C040E063E48AE383
:1001000091E00E94CD0720E044E064E483E591E0C3
:100110000E94B6020CEB12E024EB35E040E063E510
:1001200071E08BE591E00E94DD0520E042E063E4B0
:100130008BE691E00E94680220E043E063E483E7FD
:1001400091E00E94680220E042E064E48BE791E0E5
:100150000E94B60220E043E064E483E891E00E945C
:10016000B6020CE211E02CED35E041E06BE771E006
:100170008BE891E00E94DD052CED35E040E063E87E
:1001800071E08BE991E00E94DD051F910F910895C8
:100190006FEF7FEF81E090E00E947400089560E0CF
:1001A00070E08BE891E00E947F0560E070E08BE9F1
:1001B00091E00E947F051092BE01E1EBF1E0108218
:1001C000319781E0EA3AF807D1F70895EF92FF926C
:1001D0000F931F9360918D0170918E0100919D018D
:1001E00010919E01EE24FF2421E030E0F901E55555
:1001F000FE4F9081EE2DF0E0E555FE4F808198177F
:1002000008F4E22EEF2DF0E0E555FE4F80818917CE
:1002100008F4F22E2F5F3F4F2730310539F7EF2DCD
:10022000F0E0E555FE4F80818F3698F08091BD015A
:10023000882359F4EF1428F460EE7FEF0FE110E00B
:1002400004C06FE170E000EE1FEF81E08093BD011C
:1002500016C00FE110E02FEF30E04EE650E060E016
:1002600070E090E00E947906BC01EF1418F40FEFE3
:1002700010E003C08C016FEF70E01092BD018BE8BD
:1002800091E00E947F05B8018BE991E00E947F0513
:100290001F910F91FF90EF900895EF92FF920F93AF
:1002A0001F937B018C018091B9019091BA01A091BB
:1002B000BB01B091BC01A8019701281B390B4A0B67
:1002C0005B0B2F3131054105510508F44AC08AE323
:1002D00091E00E94AF07882309F443C060E08AE3FD
:1002E00091E00E94E60640E850E060E070E00E9485
:1002F000BE0620910E0130910F01F901EE54FE4F20
:1003000090E8981B90838091BE01873018F48F5F2E
:100310008093BE01E092B901F092BA010093BB0153
:100320001093BC012115310519F481E090E005C05E
:100330002630310541F48FEF9FEF909311018093A8
:1003400010010E94610080910E0190910F01209197
:10035000100130911101820F931F90930F01809330
:100360000E01E0910E01F0910F01EE0FFF1FE05022
:10037000FF4F608171818BE591E00E947F051F91A5
:100380000F91FF90EF900895CF92DF92EF92FF923E
:100390000F931F93CF93DF930E94020368EE73E0E5
:1003A0000E94A9030E94CF004BE8C42E41E0D42E46
:1003B000CBE9D1E00E9402030E940B037B018C0178
:1003C000809172018823B1F1E0916C01F0916D018F
:1003D000208130E080916B0190E028233923232B8A
:1003E00049F160EC7FEFC6010E947F0560EC7FEF72
:1003F000CE010E947F050E94020328EE33E0B8017F
:10040000A7010E941703882361F36FEF70E0C60114
:100410000E947F0561E07FEFCE010E947F050E9470
:1004200002032CED35E0B801A7010E9417038823D1
:1004300061F339C080917A018823B9F1E0917401A8
:10044000F0917501208130E08091730190E02823C4
:100450003923232B51F160EC7FEFC6010E947F0509
:1004600060EC7FEFCE010E947F050E94020328EE20
:1004700033E0B801A7010E941703882361F361E00C
:100480007FEFC6010E947F056FEF70E0CE010E94F2
:100490007F050E9402032CED35E0B801A7010E9400
:1004A0001703882361F30E94CF00C801B7010E949F
:1004B0004D018091BE01873010F00E94E6000E943D
:1004C0000203A801970164E170E00E943D0372CF2E
:1004D0001F93CF93DF93EC01122F0E94F3078F81BC
:1004E000882381F0CE010E947108EB81FC81988104
:1004F000112321F08081892B808304C08081909515
:1005000098239083DF91CF911F9108951F93CF93EC
:10051000DF93EC01122F0E94F3078F81882381F073
:10052000CE010E947108EB81FC819881112321F09A
:100530008081892B808304C080819095982390834B
:10054000DF91CF911F910895FC018781882369F085
:10055000A381B4819081662321F08C91892B8C93A7
:1005600008958C91909598239C9308951F93CF9311
:10057000DF93EC01122F0E94F3078F81882339F05B
:10058000CE010E948208612FCE010E94A402DF9159
:10059000CF911F9108951F93CF93DF93EC01122FFA
:1005A0000E94F3078F81882339F0CE010E948208D0
:1005B000612FCE010E94A402DF91CF911F91089577
:1005C0001092B200E0EBF0E0808182608083808155
:1005D0008E7F8083E1EBF0E08081877F8083808164
:1005E0008460808380818D7F808380818E7F808303
:1005F0008DE78093B300E0E7F0E080818260808344
:10060000789408958FEB91E008950E94E002089598
:100610000E94E00208952FB7F8946091C001709194
:10062000C1018091C2019091C3012FBF0895EF9243
:10063000FF920F931F937A018B016FB7F89480910B
:10064000C0019091C101A091C201B091C3016FBFDF
:1006500060E070E08E199F09A00BB10B40E050E004
:10066000281739074A075B0710F461E070E0CB01F7
:100670001F910F91FF90EF900895EF92FF920F93CB
:100680001F9379018A01AB0160E070E02FB7F89405
:100690008091C0019091C101A091C201B091C301AC
:1006A0002FBF8E199F09A00BB10B481759076A0776
:1006B0007B0760F71F910F91FF90EF9008950197CE
:1006C00039F46F5F7F4F21F48FEB91E00E940803B4
:1006D00008956FEF7FEF81E090E00E945F0308953F
:1006E0001F920F920FB60F9211242F933F934F93A7
:1006F0005F936F937F938F939F93AF93BF93EF938A
:10070000FF938091C0019091C101A091C201B0916D
:10071000C3010196A11DB11D8093C0019093C10139
:10072000A093C201B093C3010E94B7030E94EB04DF
:10073000FF91EF91BF91AF919F918F917F916F91B9
:100740005F914F913F912F910F900FBE0F901F908F
:100750001895EFB7F8942091C0013091C1014091F4
:10076000C2015091C301EFBF0E943D03089584EC84
:1007700091E00895DC012FB7F89480E090E0FC014F
:10078000EE0FFF1FEE0FFF1FE80FF91FEA0FFB1F11
:100790001382128211821082848301968031910526
:1007A00071F7A05BBF4F1D921D92FD011082118257
:1007B000128213822FBF0895DC012FB7F89480E0D6
:1007C00090E0FC01EE0FFF1FEE0FFF1FE80FF91F77
:1007D000EA0FFB1F1382128211821082848301961A
:1007E0008031910571F7A05BBF4F1D921D92FD01F5
:1007F00010821182128213822FBF0895EF92FF920E
:100800000F931F93CF93DF93EC018B01BA01FFB6D7
:10081000F894C05BDF4F5881C055D04020E0852F51
:1008200090E0FC01EE0FFF1FEE0FFF1FE80FF91F16
:10083000EC0FFD1F82819381892B39F02F5F2031CE
:1008400009F4B0C051505F70EACF503108F0AAC02F
:10085000DE01AF5ABF4F8C9190E0FC01EE0FFF1FFD
:10086000EE0FFF1FE80FF91FEC0FFD1F8281938130
:10087000892B09F48FC08C9190E0FC01EE0FFF1FD3
:10088000EE0FFF1FE80FF91FEC0FFD1F8081918114
:100890006817790708F47EC0EC9022C08D919C9176
:1008A000119768177907E0F0FD01848190E08217C5
:1008B000930711F4E42E14C0FD018481E42E482F27
:1008C000242F30E0D901AA0FBB1FAA0FBB1FA20F14
:1008D000B31FAC0FBD1FFD0182819381892BF1F6FF
:1008E000852F90E0DC01AA0FBB1FAA0FBB1FA80F2A
:1008F000B91FAC0FBD1FFD011383028311967C93BA
:100900006E935483FFEFEF1621F12E2D30E0F901A5
:10091000EE0FFF1FEE0FFF1FE20FF31FEC0FFD1F87
:10092000848190E08217930721F08481FD01848304
:1009300005C0CF5ADF4F5883C155D040F901EE0FA3
:10094000FF1FEE0FFF1FE20FF31FEC0FFD1F54837D
:1009500029C09E01205B3F4FF901808190E0FC019E
:10096000EE0FFF1FEE0FFF1FE80FF91FEC0FFD1F2B
:1009700082819381892B29F0F9018081FD01848393
:1009800005C0CF5ADF4F5883C155D040C05BDF4F01
:10099000588308C0C05BDF4F4881C055D040EE246B
:1009A000EA948ECFFFBEDF91CF911F910F91FF9000
:1009B000EF900895019739F46F5F7F4F21F484EC35
:1009C00091E00E94DC0308956FEF7FEF81E090E0FB
:1009D0000E94DA0408958F929F92AF92BF92CF92B5
:1009E000DF92EF92FF920F931F93CF93DF935C01FF
:1009F0000E9402030E940B039B01AC01F501EE5A19
:100A0000FF4F80819181A281B38179018A01E81A27
:100A1000F90A0A0B1B0B09F44BC080819181A2815A
:100A2000B381281739074A075B0728F40894E108BF
:100A3000F108010911092083318342835383F501B1
:100A4000E05BFF4FC0804F0124C0DC80888199812A
:100A5000A0E0B0E0E816F9060A071B0788F0EA8173
:100A6000FB811B821A8219821882CC82D401DC920B
:100A7000A081B1812D913C91CF01F901099506C06A
:100A8000888199818E199F0999838883CD1481F07B
:100A9000CD2C8C2D90E0EC01CC0FDD1FCC0FDD1F99
:100AA000C80FD91FCA0DDB1D8A819B81892B69F66E
:100AB000DF91CF911F910F91FF90EF90DF90CF903A
:100AC000BF90AF909F908F900895FC0187818823FD
:100AD00069F0A381B4819081662321F08C91892BE8
:100AE0008C9308958C91909598239C93089561E040
:100AF0000E94A402089560E00E94A4020895CF928B
:100B0000DF92EF92FF920F931F93CF93DF93EC014D
:100B10000E94AB086C018C81882309F443C0ED80EE
:100B2000FE800F8118850E94020324E130E0B801A5
:100B3000A7010E9417038823A9F18B85882321F040
:100B4000D094C194D108D3942C853D858E859F8502
:100B50008C01020F131F281B390B4FEF50E061E08F
:100B60007FEFC6010E9479068C01FFB6F894898553
:100B70009A850E947705C80164E170E00E94F80838
:100B8000CB0168E070E00E94500689859A850E943A
:100B90007B05FFBE0E9402030E940B036D837E83D0
:100BA0008F8398878A819B81DF91CF911F910F91CD
:100BB000FF90EF90DF90CF900895AF92BF92DF92B9
:100BC000EF92FF920F931F93CF93DF93EC015B01A2
:100BD000D42E79010E94920886E191E0998388835E
:100BE000DB86FD86EC861F870E87F50187818823CB
:100BF00089F0BA86A986C5010E947B050E9402037E
:100C00000E940B036D837E838F839887CE010E94A1
:100C1000A70802C01A861986DF91CF911F910F9104
:100C2000FF90EF90DF90BF90AF900895AF92BF928A
:100C3000DF92EF92FF920F931F93CF93DF93EC011C
:100C40005B01D42E79010E94920886E191E099839C
:100C50008883DB86FD86EC861F870E87F5018781FA
:100C6000882389F0BA86A986C5010E947B050E9467
:100C700002030E940B036D837E838F839887CE01CE
:100C80000E94A70802C01A861986DF91CF911F9192
:100C90000F91FF90EF90DF90BF90AF90089508956F
:100CA000CF93DF93CDB7DEB722970FB6F894DEBFB0
:100CB0000FBECDBF9A83898389819A819C01629FEF
:100CC000C001639F900D729F900D112403C0898114
:100CD0009A8101979A83898389819A81892BB9F7AF
:100CE00022960FB6F894DEBF0FBECDBFDF91CF9135
:100CF00008954F925F926F927F928F929F92AF92E0
:100D0000BF92CF92DF92EF92FF920F931F932B012E
:100D10005A0139017801E21AF30A0027F7FC00951D
:100D2000102F9C01261B370B442737FD4095542F6D
:100D3000C801B7010E94D908A418B508CC24B7FC93
:100D4000C094DC2CA60195010E942D09882477FC13
:100D50008094982C620E731E841E951EC3011F91F1
:100D60000F91FF90EF90DF90CF90BF90AF909F904A
:100D70008F907F906F905F904F90089568177907DC
:100D80000CF4BC01461757070CF4BA01CB010895C7
:100D9000CF93DF93DC01EC018F81882319F420E0ED
:100DA00030E00EC0ED01E981FA8120818C9130E0C4
:100DB00090E0282339232115310511F021E030E09E
:100DC00081E0822790E0DF91CF9108951F93CF9328
:100DD000DF93EC01162FE881F9810190F081E02D7D
:100DE000099524E630E0829FB001839F700D929FA9
:100DF000700D112480E090E022E831E040E050E006
:100E00000E940B09C9011123D1F1688D67FF0DC044
:100E1000188EFE0120E030E0918B808B2F5F3F4FDA
:100E200032962830310559F1F7CFE62FFF27E7FD3D
:100E3000F095EE0FFF1FEC0FFD1F318B208B6F5FC6
:100E40006770688FFE0120E030E040E050E060E035
:100E500070E080899189A0E0B0E0280F391F4A1F17
:100E60005B1F6F5F7F4F32966830710591F783E0AB
:100E700056954795379527958A95D1F7C901DF9102
:100E8000CF911F910895FF920F931F93CF93DF93FC
:100E9000EC018985882309F45AC0E881F98104802E
:100EA000F581E02DCE010995882309F450C0EF812A
:100EB000F88580819A81892B8083ED81FE819081E4
:100EC0008A81809589238083FFB6F894ED81FE8125
:100ED00080819A81892B808368E070E081E090E0D6
:100EE0000E945006ED81FE8190818A818095892340
:100EF0008083EF81F88590818A8180958923808322
:100F00008E010E5F1F4FC8010E94C8068823D9F7C3
:100F100040E050E002C04F5F5F4FEB81FC812081D9
:100F20008A8130E090E028233923232BA1F7FFBEEC
:100F300023E0569547952A95E1F75F874E870E94F3
:100F400002030E940B036A877B878C879D878E85AF
:100F50009F85DF91CF911F910F91FF900895EF92A0
:100F6000FF920F931F93FC01E284F384048515859F
:100F7000E114F1040105110511F481E008C00E949B
:100F8000020322E330E0B801A7010E94170390E0BA
:100F90001F910F91FF90EF9008950F931F938C0175
:100FA0000E94CA0880E291E0F80191838083128652
:100FB0001386148615868FEF808F1F910F910895E9
:100FC0000F931F938C010E94CA0880E291E0F80100
:100FD0009183808312861386148615868FEF808F07
:100FE0001F910F910895FC0181E090E002C0880FED
:100FF000991F4A95E2F7808381E08783643419F171
:1010000065342CF4623449F0633451F511C0633611
:1010100079F06436C1F0623619F584E290E0968387
:10102000858383E290E09283818385E290E015C01E
:1010300087E290E09683858386E290E092838183C5
:1010400088E290E00AC08AE290E09683858389E294
:1010500090E0928381838BE290E094838383089570
:1010600017820895FC0181E090E002C0880F991F6B
:101070004A95E2F7808381E08783643419F165340F
:101080002CF4623449F0633451F511C0633679F0C1
:101090006436C1F0623619F584E290E09683858368
:1010A00083E290E09283818385E290E015C087E23D
:1010B00090E09683858386E290E09283818388E244
:1010C00090E00AC08AE290E09683858389E290E00E
:1010D000928381838BE290E09483838308951782C7
:1010E0000895CF93DF93DC01EC018F81882339F0E1
:1010F000ED81FE8190818C91809589238083DF91A1
:10110000CF910895CF93DF93DC01EC018F81882389
:1011100031F0ED81FE8180819C91892B8083DF916C
:10112000CF910895FC018AE291E09183808313823C
:10113000128214820895FC018AE291E091838083F7
:101140001382128214820895FC011482089521E012
:10115000FC01248308950F931F938C01CB014FEF63
:1011600050E061E07FEF0E94BE06F8019383828326
:101170001F910F9108950F931F938C0120E0029609
:101180000E94860284E391E0F801918380831F919D
:101190000F9108950F931F938C0120E002960E94F7
:1011A000860284E391E0F801918380831F910F917F
:1011B0000895629FD001739FF001829FE00DF11DA1
:1011C000649FE00DF11D929FF00D839FF00D749FC1
:1011D000F00D659FF00D9927729FB00DE11DF91F6D
:1011E000639FB00DE11DF91FBD01CF0111240895CA
:1011F00097FB092E07260AD077FD04D049D006D0E8
:1012000000201AF4709561957F4F0895F6F7909538
:1012100081959F4F0895A1E21A2EAA1BBB1BFD01C9
:101220000DC0AA1FBB1FEE1FFF1FA217B307E407C5
:10123000F50720F0A21BB30BE40BF50B661F771F1D
:10124000881F991F1A9469F76095709580959095FD
:101250009B01AC01BD01CF01089597FB092E052626
:101260000ED057FD04D0D7DF0AD0001C38F45095BB
:101270004095309521953F4F4F4F5F4F0895F6F7BA
:1012800090958095709561957F4F8F4F9F4F0895F2
:10129000AA1BBB1B51E107C0AA1FBB1FA617B7079C
:1012A00010F0A61BB70B881F991F5A95A9F78095B8
:1012B0009095BC01CD010895EE0FFF1F0590F491AC
:0612C000E02D0994FFCFB0
:1012C60001FF56FFABFF00005500AA00FF00040017
:1012D6000100000000007F05A708A4080000000028
:1012E6004307E606AF07000000004F06A708A4085C
:0A12F600000000004F064F064F06EF
:00000001FF
